:020000040000fa
:08000000a2060400000000004c
:020000040000fa
:020000040002f8
:04afe000dfff00008f
:020000040000fa
:020000040002f8
:04afe400ffff00006b
:020000040000fa
:020000040002f8
:04afe80078ff0000ee
:020000040000fa
:020000040002f8
:04afec007dff0000e5
:020000040000fa
:020000040002f8
:04aff00078ff0000e6
:020000040000fa
:1000080000000000000000000000000000000000e8
:100018009a06000000000000000000000000000038
:10002800000000000000000000000000040a0000ba
:1000380000000000000000000000000000000000b8
:10004800460a00000000000000000000ce0a000080
:100058003a0b0000660b00000000000000000000e2
:100068000000000000000000000000000000000088
:100078000000000000000000000000000000000078
:10008800000000000000000000000000720a0000ec
:10009800a00a0000000000000000000000000000ae
:1000a8000000000000000000000000000000000048
:1000b8000000000000000000000000000000000038
:1000c8000000000000000000000000000000000028
:1000d8000000000000000000000000000000000018
:1000e8000000000000000000000000000000000008
:1000f80000000000000000000000000000000000f8
:1001080000000000000000000000000000000000e7
:1001180000000000000000000000000000000000d7
:1001280000000000060b00000000000000000000b6
:1001380000000000000000000000000000000000b7
:1001480000000000000000000000000000000000a7
:100158000000000000000000000000000000000097
:100168000000000000000000000000000000000087
:100178000000000000000000000000000000000077
:100188000000000000000000000000000000000067
:100198000000000000000000940b0000c00b0000ed
:1001a800ec0b000000000000000000000000000050
:1001b8000000000000000000000000000000000037
:1001c8000000000000000000000000000000000027
:1001d8000000000000000000000000000000000017
:1001e8000000000000000000000000000000000007
:1001f80000000000000000000000000000000000f7
:1002080000000000000000000000000000000000e6
:1002180000000000000000000000000000000000d6
:1002280000000000000000000000000000000000c6
:1002380000000000000000000000000000000000b6
:1002480000000000000000000000000000000000a6
:100258000000000000000000000000000000000096
:100268000000000000000000000000000000000086
:0c0278000000000000000000000000007a
:020000040000fa
:10040000803e2000030007008100e900fcff3a0065
:1004100000000600831f7800c20320000400bc0017
:1004200066015100e0815900f23fb1000380b10044
:1004300006003500ee03090000000000423fb10055
:100440000380b100fbff3d001200b000223fb0006e
:10045000020035000280090000000000cf01780092
:10046000000006000001eb00869fbe00889fbe00d2
:100470008a9fbe008c9fbe00820578000004be00eb
:10048000e00107000800be006420e1000700390019
:1004900002003a00f1ff2f00f0ff27000160a000ea
:1004a0001202200002918800560037006120e1000e
:1004b00003003a000b00a70001f8230051003700a9
:1004c00001f0a10002002100936424005200070003
:1004d0000800be0005003500b2fd2000930c24008a
:1004e00004002000690007000004be000005eb00c6
:1004f0000b00a6004f0dde0001f0a1000004be00bd
:1005000032982f0023ea23000f0107000001eb00bf
:10051000030020000b00a70003f82300ac00070035
:100520003e0107000000a7000a00a20080010700aa
:100530000b00e000030032000200200003f0230063
:10054000a200070001f0a2000006be000200200089
:1005500093042400fc0007000801be009c00070073
:10056000809fbe000c00be0022a22a00d3a7230059
:10057000f50007004f01be00950007000004be0013
:1005800001f0a100020020000398230022000700d0
:100590000800be00190035000001be00ea00070097
:1005a0000006be00b2c52900e3622300e600070092
:1005b00022222b00f3942b00850007000c01be00c3
:1005c000e1000700e273280083c0230080000700d9
:1005d0000c01be00dc00070042aa2a00a3e22b00a7
:1005e0007b0007000c01be00d70007000801be0019
:1005f000d50007000801be00750007000a00a7002b
:1006000001f0a2004f06be004f05be004f04be0021
:100610004f03be000000060014002000889fbe00ab
:100620008a9fbe00841f78006e0107004f0078008b
:1006300011003300f0ff2f00838f6c0006003b0099
:10064000040565000a00a7000800370009f0a600ad
:100650001000200008003700820f5400838f5c00d8
:10066000030039001000200001003e0000002000bf
:1006700009f0a7000000ea004f05be004f04be00cd
:100680000000e0000000060014002000869fbe006d
:10069000889fbe008a9fbe008c9fbe004f26dd0053
:1006a00050010700920133006120e1004300320055
:1006b0006250e10041003e003e0039006420e1004c
:1006c0003c003200058255000f003b000402e800a8
:1006d00038003a00800f5300818f5b0035003400f2
:1006e0000800be0003f0a10001f0a60003f0a00086
:1006f0000cf0a70036000700860137000603430010
:1007000087834b000c4646000005530081855b0043
:10071000020033000a03be000c00a0000402e9003e
:10072000f6ff3b00850578000602430087824b00f8
:1007300004003a006000b80009f0a70001f0a00032
:10074000740137000002520081825a000704e00061
:10075000040033000603430087834b008b05e90048
:10076000faff3700090578000604be000203be0048
:100770006011b80038010700e00f5200e08f5a0006
:100780000700350002003c000c08a3000400320002
:100790000601be0003f0a0000cf0a7000c0007004b
:1007a0000a85680001f0a1000af0a70001f0a0008e
:1007b000580137000800be00560137001002200023
:1007c0000cf0a600009188005701370003f0a2004a
:1007d000869fbe00889fbe008a9fbe008c9fbe0081
:1007e00000010700420133006450e1004f00320075
:1007f0006420e1005200320003826c0007003b00dd
:100800000905d0000306d000820f54000c065d00dd
:1008100002003900020032008901780003067800e6
:100820008582550004003d000003fd008103fd00aa
:100830008502ea008b854200840f720002003b00b3
:1008400060001000e08018006011b8000005eb00a7
:100850007a28e1000a00390006007800c75ddd0053
:10086000f707b200878075002d0037008281710084
:100870000a017800610560008180d1000080d3000a
:100880008502e900f9ff3b00060440008784480028
:1008900002003b0060041400e0841c000988a300ef
:1008a000070032008a817100828171006101640059
:1008b0008904d1000884d3008b05e80017003700b5
:1008c0000978a30013003a000b00e0001300340085
:1008d0008b05e9000804440089844c000a44740034
:1008e0000978a3000d003a000b00e0000700340077
:1008f0008b05e9000804440089844c0001003a009b
:100900000b0020000978a300f7ff32000001eb0084
:1009100002003700828171000a017800ce000700d2
:100920000cf0a70001f0a000fa0037006420e100fd
:1009300002003a00838f6c00fb0033000801be0008
:100940000200be00f3003700869fbe00889fbe00f5
:100950008a9fbe008c9fbe00a2000700e400330007
:1009600003866c006450e100240032006420e10042
:10097000270032006150e100220032006120e100d6
:10098000210032008b854200eb07b1000134b80032
:10099000003ab8000804420089844a00013ab800cd
:1009a0000030b8008880400009014a00040033008c
:1009b0000000400081804800020149008b05e900e9
:1009c000c909dd008301700001003200130020001e
:1009d000c814de004814dd004709de001200b20032
:1009e000c808de00088470009b00070001f0a10029
:1009f0000cf0a70001f0a000c60037006120e10064
:100a0000c90032000801be000200be00f7ff370037
:100a10006150e100fcff3a00c3003700829fbe0036
:100a20000001be00770007000470a70003f0a100da
:100a30006509b100180032000e0035006828e10099
:100a400007003500f0ff2f00f1ff27000300e00052
:100a500015003b00010028004f01be00000005000a
:100a600000004000818048008502e900fcff3a0058
:100a700009003700f88f420003003c008000eb00c3
:100a80004f01be00000005008100d1000080d300ae
:100a90008502e800fcff3a000300e00002003b0092
:100aa00060001000e08018004f01be00000006004a
:100ab000829fbe000001be00520007000470a70024
:100ac00003f0a10003f8a30015003a006509b10086
:100ad000110032000a0035006928e10003003500ea
:100ae000010028004f01be0000000500000040008a
:100af000818048008502e900fcff3a0006003700cb
:100b0000f88f4200060035008100d1000080d3003c
:100b10008502e800fcff3a004f01be00000006001d
:100b20008000eb004f01be00000005008000eb00dc
:100b3000829fbe00889fbe008a9fbe00010578008c
:100b40000100e0000400350008003c000000e00067
:100b5000200032000500370060001000e08018001f
:100b600002003b0001f024001a0037000004be0020
:100b70006011b8006b0920000982cf000200390023
:100b80000882cf000441b000694252000e003200da
:100b900008003b0082817100610164008904d1007a
:100ba0000884d3008b05e8000442e800f9ff3a000e
:100bb000050037000804440089844c008b05e900d7
:100bc0000442e900fbff3a00230007000af0a700f7
:100bd00001f0a0004f05be004f04be004f01be0053
:100be000000006000004be00060007000003be006f
:100bf0000405be000200be0002000700844f75001d
:100c000000000600c70ade00f107b200f50fb200cf
:100c100008003200e1cf4200020032000170a00063
:100c200024000500810f7000010032000408050057
:100c300044000500810f700002003a001400050016
:100c40008502e9000000400081c04800fcff3b0035
:100c50000170a00024000500810020006180550083
:100c60000b003d000b00200061fe2f000100e100a1
:100c70001d00340082817100610164008904d1008b
:100c80000884d3000000e800faff3a007100200059
:100c9000610064000300700002006000090032007f
:100ca00061044400e0844c000988a500050032007e
:100cb0008b05e8006808e10002003a008904d100d1
:100cc0000884d300f20f20000258e10005003d0027
:100cd000c75ddd00f907b200898075000800780063
:100ce000000006000bf827008b00780000000500cc
:100cf0000200be006450e100050036006420e100ff
:100d0000020036000968a30001003a000800be0096
:100d10000160a0004f06be004f05be004f04be009c
:100d20004f03be0000000600f0ff2f00f1ff270078
:100d3000f8ff37000020ef000220ef00c088a90074
:100d4000004006000f002100b02e210000018800a5
:100d5000000000000000eb00000778000c00090014
:100d6000002f78000007eb005420ef000e2eef005c
:100d70001e2eef000000eb00a1212100e51d09005f
:100d80008018780040a7a900a10020009cfd070062
:100d9000e0022000303a880044e7a90044c7a900d7
:100da0004407a9004427a9004447a9004467a900b3
:100db0004487a900300020000600fc0031742000a8
:100dc00082072000a3092000824878008348780029
:100dd00080487800113a8000618070000600fc00b5
:100de00021742000620420007305200082487800ee
:100df00083487800804878004427ef00e002200014
:100e0000303a8800300020000d00fc0031742000d2
:100e100082072000a30920008248780083487800d8
:100e20008048780000002000217420006204200027
:100e30007305200082487800834878008048780055
:100e400042a7ae00feff3700813e20006cfd070088
:100e500010c0b30086e6b70090c2b300c4e6b70086
:100e6000000220000070880000702500807088005b
:100e700010eea90010cea90010aea900008ea900a6
:100e8000108ea900000ea900002ea900100ea900c6
:100e9000102ea900ae04070094050700cd06070038
:100ea000af0607000000eb0081772100ff0009007a
:100eb000805878005a72ef005b72ef003a32ef0010
:100ec0003c32ef000080eb00417721000100090077
:100ed000801878002632ef003832ef004188a800f1
:100ee00041a8a90041c8a80000a1ef0000582200b5
:100ef0001008880004a1a9000481a80005e1a80049
:100f00000068a9002068a8001061a8001021a900ad
:100f100011e1a80011a1a90010a1a8001081a8004a
:100f20000621ef000a21ef000ca1ef000ea1ef0057
:100f30004408a9004428a9004448a9000108a900c0
:100f40002108a8002002a9002022a9002042a9000f
:100f500020a2a9002062a9002082a90020e2a90005
:100f60002102a9002122a900700720004011880059
:100f700022a2a90022c2a90022e2a90021e2a8001f
:100f80002182a9004588a90045a8a80045c8a80055
:100f90002168a8002828a8002bc8a9002be8a900d0
:100fa0002c08a9000bc8a9000be8a9000c08a9008f
:100fb00001eca90001aca900016ca900014ca90039
:100fc000012ca900010ca90000eca900008ca900cb
:100fd00000aca90000cca900000ca900002ca900bd
:100fe000004ca900006ca900202cef00402cef0061
:100ff000602cef000010200020608800020ca90087
:10100000022ca800024ca900f007200030618800e3
:10101000f007200030628800f0072000306388006d
:10102000282cef00482cef00682cef000010200067
:101030005060880023eca80023cca80023aca900b2
:10104000238ca900236ca900234ca900232ca90000
:10105000230ca900222ca90043eca80043cca80033
:1010600043aca900438ca900436ca900434ca900e0
:10107000432ca900430ca90063eca80063cca80092
:1010800063aca900638ca800636ca900634ca90041
:10109000dabc2a001b32240030002c00fa608800e1
:1010a000fb60880020618800dabc2a001b32240023
:1010b00000002c00fa608800fb6088001061880046
:1010c000dabc2a001b32240030002c00fa608800b1
:1010d000fb60880020628800dabc2a001b322400f2
:1010e00000002c00fa608800fb6088001062880015
:1010f000dabc2a001b32240030002c00fa60880081
:10110000fb60880020638800dabc2a001b322400c0
:1011100000002c00fa608800fb60880010638800e3
:10112000a80037003f003700002020000061880041
:10113000002020000062880000202000006388005a
:10114000020ca900022ca800024ca80004acef007d
:1011500028acef0048acef0068acef00262cef00a5
:10116000462cef00662cef000aacef0023eca80041
:1011700023cca90043eca80043cca90063eca80051
:1011800063cca900dabc2a001b32240030002c00fa
:10119000fa608800fb60880020618800dabc2a00c1
:1011a0001b32240000002800fa608800fb608800e1
:1011b00010618800dabc2a001b32240030002c00a9
:1011c000fa608800fb60880020628800dabc2a0090
:1011d0001b32240000002800fa608800fb608800b1
:1011e00010628800dabc2a001b32240030002c0078
:1011f000fa608800fb60880020638800dabc2a005f
:101200001b32240000002800fa608800fb60880080
:101210001063880011eea90011aea900116ea9009b
:101220006800370036003700001020000061880099
:101230000010200000628800001020000063880079
:10124000020ca900022ca800024ca8000a2cef00f6
:101250000040200020608800282cef005055250019
:1012600040628800a0aa2a0040638800dabc2a00f5
:101270001b32240030002c00fa608800fb608800dc
:1012800020618800dabc2a001b32240000002c00f8
:10129000fa608800fb60880010618800dabc2a00d0
:1012a0001b32240030002c00fa608800fb608800ac
:1012b00020628800dabc2a001b32240000002c00c7
:1012c000fa608800fb60880010628800dabc2a009f
:1012d0001b32240030002c00fa608800fb6088007c
:1012e00020638800dabc2a001b32240000002c0096
:1012f000fa608800fb6088001063880031003700c6
:10130000300037000010200000618800001020002d
:1013100000628800020ca900022ca800024ca80060
:101320000a2cef0004acef00282cef000000240092
:1013300040628800dabc2a001b32240030002c00f6
:10134000fa608800fb60880020618800dabc2a000f
:101350001b32240000002c00fa608800fb6088002b
:1013600010618800dabc2a001b32240030002c00f7
:10137000fa608800fb60880020628800dabc2a00de
:101380001b32240000002c00fa608800fb608800fb
:1013900010628800dabc2a001b32240030002c00c6
:1013a000fa608800fb60880020638800dabc2a00ad
:1013b0001b32240000002c00fa608800fb608800cb
:1013c00010638800218ca900418ca900618ca900c0
:1013d000216ca900416ca900616ca900214ca900f5
:1013e000414ca900614ca90020eca80040eca800e9
:1013f00060eca8003e2cef005e2cef007e2cef008e
:1014000001eca80016013700ff3ffc004200f80085
:101410003600f8004400f8008e1f78000e0020000f
:101420000d000900be1f78003200f8000100fc002a
:101430000068a9000021ef002fd2bf000080fb0050
:101440003061880031d2bf000080fb00306288002c
:1014500033d2bf000080fb00306388006e72ec0066
:10146000ff3ffc003200f900ae0120000d00090032
:101470004f1778004f0778004400f9003600f90054
:101480004200f9000100fc0000400600ff3ffc00a4
:101490004200f8003600f8004400f8008e1f780083
:1014a0000e0020000d000900be1f78003200f80079
:1014b0000100fc000108a900ff3ffc003200f90018
:1014c000ae0120000d0009004f1778004f0778008b
:1014d0004400f9003600f9004200f9000100fc0068
:1014e00000400600ff3ffc004200f8003600f80014
:1014f0004400f8008e1f78000e0020000d00090047
:10150000be1f78003200f8000100fc000368a9004b
:101510001421ef00ff3ffc003200f900ae01200073
:101520000d0009004f1778004f0778004400f900bc
:101530003600f9004200f9000100fc0000400600fe
:10154000ff3ffc004200f8003600f8004400f800bd
:101550008e1f78000e0020000d000900be1f7800cd
:101560003200f8000100fc000388a9001821ef00f8
:10157000ff3ffc003200f900ae0120000d00090021
:101580004f1778004f0778004400f9003600f90043
:101590004200f9000100fc0000400600ff3ffc0093
:1015a0004200f8003600f8004400f8008e1f780072
:1015b0000e0020000d000900be1f78003200f80068
:1015c0000100fc000168a9005a72ec005ad2bf0069
:1015d0008080fb00301180008277210080707900cc
:1015e000ff3ffc003200f900ae0120000d000900b1
:1015f0004f1778004f0778004400f9003600f900d3
:101600004200f9000100fc0000400600ff3ffc0022
:101610004200f8003600f8004400f8008e1f780001
:101620000e0020000d000900be1f78003200f800f7
:101630000100fc000828a9002242ae00000037008b
:101640002222af002222a900ff3ffc003200f90055
:10165000ae0120000d0009004f1778004f077800f9
:101660004400f9003600f9004200f9000100fc00d6
:1016700000400600ff3ffc004200f8003600f80082
:101680004400f8008e1f78000e0020000d000900b5
:10169000be1f78003200f8000100fc000188a9009c
:1016a000ff3ffc003200f900ae0120000d000900f0
:1016b0004f1778004f0778004400f9003600f90012
:1016c0004200f9000100fc0000400600ff3ffc0062
:1016d0004200f8003600f8004400f8008e1f780041
:1016e0000e0020000d000900be1f78003200f80037
:1016f0000100fc0001a8a9002003a900ff3ffc0095
:101700003200f900ae0120000d0009004f177800eb
:101710004f0778004400f9003600f9004200f90054
:101720000100fc0000400600ff3ffc004200f80002
:101730003600f8004400f8008e1f78000e002000ec
:101740000d000900be1f78003200f8000100fc0007
:101750000bc8a900ff3ffc003200f900ae012000d9
:101760000d0009004f1778004f0778004400f9007a
:101770003600f9004200f9000100fc0000400600bc
:10178000ff3ffc004200f8003600f8004400f8007b
:101790008e1f78000e0020000d000900be1f78008b
:1017a0003200f8000100fc000be8a900ff3ffc003c
:1017b0003200f900ae0120000d0009004f1778003b
:1017c0004f0778004400f9003600f9004200f900a4
:1017d0000100fc0000400600ff3ffc004200f80052
:1017e0003600f8004400f8008e1f78000e0020003c
:1017f0000d000900be1f78003200f8000100fc0057
:101800000c08a900ff3ffc003200f900ae012000e7
:101810000d0009004f1778004f0778004400f900c9
:101820003600f9004200f9000100fc00004006000b
:101830005bd2bf005a52e300070032005b72ec003b
:101840005bd2bf000080fb008177210060c0780080
:101850005cf2b700010037005cf2ef000000060008
:1018600050088000e091880030088000d091880006
:10187000efff070060ceb3005c52b50006003900f0
:10188000e0cfb3005c52b500010039000100370021
:101890005d72ef00450137005cf2ae0037003700a3
:1018a0005d72ef0050c8b3005c52e30005003a00df
:1018b0005cd2bf005df2b7005ef2ef005ff2ef00b6
:1018c0002d00370050c9b3005c52e30005003a0018
:1018d0005cd2bf005df2b70060f2ef0061f2ef0092
:1018e0002500370050cab3005c52e30005003a00ff
:1018f0005cd2bf005df2b70062f2ef0063f2ef006e
:101900001d00370050cbb3005c52e30005003a00e5
:101910005cd2bf005df2b70064f2ef0065f2ef0049
:101920001500370050ccb3005c52e30004003a00cd
:101930005cd2bf005df2b70066f2ef000e00370028
:1019400050cdb3005c52e30004003a005cd2bf000b
:101950005df2b70067f2ef000700370050ceb3002a
:101960005c52e30004003a005cd2bf005df2b700b5
:1019700068f2ef0069f2ef000c0137005d52e200ff
:1019800002003a00090137000801370050c8b300cf
:101990005d52e30048003a0000e0ef005e52e300d1
:1019a00003003a005cd2bf005ef2b700410037008e
:1019b0005cd2bf005ff2b70090c1b3005e52e3009b
:1019c0002d003a005f52e20012003a0014cea90046
:1019d00005e1a900f007200030618800f007200031
:1019e00030628800f0072000306388007172ef00d9
:1019f0003612a9002612ae000400370074b7ef00bb
:101a000076b7ef006c12a8002612a900140ea900e8
:101a100018003700022eae00160037003612a8005c
:101a200005e1a800020021005fd2bf000080fb009a
:101a30000200b8000001be00a2bb8800b3bb880052
:101a4000a2bb8000b3bb8000d0918000e1918000f8
:101a500002004000838048000001be00a2bb880055
:101a6000b3bb88002612a8006c12a800140ea900af
:101a7000142ea8000e00370080c7b3005e52e300aa
:101a800002003a0014aea9000900370090c7b30065
:101a90005e52e30002003a00048ea9000400370001
:101aa000a0c7b3005e52e30001003a00148ea90003
:101ab0005ef2ef00bd00370050c9b3005d52e30095
:101ac0006e003a0000e0ef006052e30003003a00cd
:101ad0005cd2bf0060f2b700670037005cd2bf0085
:101ae00061f2b7006152e20024003a0090c1b300f5
:101af0006052e30012003a0014cea90005e1a900eb
:101b0000f007200030618800f00720003062880074
:101b1000f0072000306388007172ef003612a900d0
:101b20002612ae000400370074b7ef0076b7ef005e
:101b30006c12a8002612a900140ea9000e0037008e
:101b400080c7b3006052e30002003a0014aea9005f
:101b50000900370090c7b3006052e30002003a006a
:101b6000048ea90004003700a0c7b3006052e30050
:101b700001003a00148ea9003e00370090c1b30066
:101b80006052e30021003a0061d2bf0072f2b70058
:101b9000022eae001900370014cea80072d2bf008a
:101ba0000080fb0000004000412721006080780099
:101bb0001008880005e1a8000068a9002068a800b6
:101bc0006e72ef0072d2bf000080fb000000d100f7
:101bd0000044b00071f2b7003612a9002612ae0020
:101be0000400370074b7ef0076b7ef006c12a8005e
:101bf0002612a900140ea8000300370014cea90075
:101c0000140ea9007172ef001a00370080c7b300ec
:101c10006052e30006003a00022eae0002003700d8
:101c200014aea8000100370014aea900110037005f
:101c300090c7b3006052e30006003a00022eae00e7
:101c400002003700048ea80001003700048ea900ae
:101c500008003700a0c7b3006052e30005003a0057
:101c6000022eae0002003700148ea80001003700db
:101c7000148ea90060f2ef004c00370050cab30088
:101c80005d52e3001b003a0000e0ef006252e30007
:101c900003003a005cd2bf0062f2b70014003700c4
:101ca0005cd2bf0063f2b70090c1b3006252e300a0
:101cb0000e003a0012ceae000c0037006e72ef003c
:101cc00063d2bf000080fb000000d1000044b000e0
:101cd00071f2b70063d2bf000080fb00000040003b
:101ce00041272100608078001008880062f2ef0030
:101cf0002e00370050cbb3005d52e3000b003a00da
:101d000000e0ef006452e30003003a005cd2bf0041
:101d100064f2b700040037005cd2bf0065f2b70080
:101d2000dc00070064f2ef002000370050ccb30065
:101d30005d52e30007003a0000e0ef006652e30066
:101d400003003a005cd2bf0066f2b70066f2ef0013
:101d50001600370050cdb3005d52e30007003a0093
:101d600000e0ef006752e30003003a005cd2bf00de
:101d700067f2b70067f2ef000c00370050ceb300f7
:101d80005d52e30009003a0000e0ef006852e30012
:101d900003003a005cd2bf0068f2b70003003700ce
:101da0005cd2bf0069f2b70068f2ef006c12af00be
:101db0009b00070010c0b3006b52b5002500310036
:101dc000d2918000e39180001092800021928000e7
:101dd000800f5100818f59001200390045f2a80090
:101de0006b52e2000e003a0014cea90005e1a900f2
:101df000f007200030618800f00720003062880082
:101e0000f0072000306388007172ef0074b7ef00b4
:101e100076b7ef003612a9002612a900142ea900e9
:101e20007f0007003df2ae00090037000621ef00f9
:101e30000a21ef003a32ef003c32ef000080eb0065
:101e400041772100010009008018780084fe3700e6
:101e5000040037003df2ae00020037000621ef001b
:101e60000a21ef006dd2bf006e52e3006500320020
:101e70003612af00340037006ed2bf000080fb0086
:101e8000000040004137210060807800d090880039
:101e900011272100914078008100fb00d090800044
:101ea0000088b90040918800000028002812b40082
:101eb000709188006ed2bf00b040b0006ff2b700e2
:101ec0006fd2bf000080fb000000400041372100be
:101ed00060807800d0908800112721009140780020
:101ee0008100fb00d09080000088b90050918800ec
:101ef000000028002a12b400809188006ed2bf0032
:101f00006041b00070f2b70070d2bf000080fb00eb
:101f1000000040004137210060807800d0908800a8
:101f200011272100914078008100fb00d0908000b3
:101f30000088b90060918800000028002c12b400cd
:101f4000909188002d0037002612ae002500370042
:101f50006ed2bf000080fb0000004000413721002e
:101f6000608078004700dd00409188000000280074
:101f70002812b40070918800b0c0b3006e52b50052
:101f80006ff2b7006fd2bf000080fb00000040007e
:101f900041372100608078004700dd0050918800c3
:101fa000000028002a12b4008091880060c1b300ac
:101fb0006e52b50070f2b70070d2bf000080fb0017
:101fc0000000400041372100608078004700dd00bc
:101fd00060918800000028002c12b40090918800c5
:101fe00006003700000028007091880000002800db
:101ff0008091880000002800909188006ed2bf0078
:102000006df2b700020eaa00000ea9003c32af002c
:1020100014eea8003c32ae0014eea90010fe37000a
:102020006bf2ef0045f2a8002432ef00209180000f
:10203000c200dd0040772100008040001000be009b
:102040000001be001092800021928000800f51009c
:10205000818f59000900310020918000c200dd000d
:1020600040772100008040001000be0010928800e0
:102070002192880024d2bf006bf2b7002432ec001a
:1020800021918000e18f5000e8ff3a006c12a90016
:102090000000060020c4b3006452e3001a003a00b6
:1020a0006552e20016003a002432ef002412e200ea
:1020b00009003e0020918000c200dd004077210031
:1020c00000814000f0ff2f00f1ff2f000089be00cb
:1020d0002432ec00f5ff39002632ef006c12a80024
:1020e00014cea90014aea900048ea900148ea90074
:1020f000042ea900142ea9006e72ef000100370013
:10210000042ea80010003700b0c7b3006452e300eb
:102110000d003a0014cea9000008200030618800ac
:10212000000820003062880000082000306388002a
:1021300074b7ef0076b7ef002632ef0014aea900b7
:10214000048ea900148ea90064f2ef0000000600be
:1021500074b6ef00101a2f00b0b3880010412e00a3
:10216000c0b3880040742d00d0b38800f0b22c00ba
:10217000e0b3880070fc2b00f0b3880030502b00d7
:1021800000b48800a0ad2a0010b4880030142a00e2
:1021900020b488006083290030b48800b0fa280099
:1021a00040b48800a079280050b48800c000200006
:1021b0002091880021918000f78f50000e003e0092
:1021c000c00020002412b500000678000c0646006e
:1021d0004067210060007e004100de002291800007
:1021e0004111dd0041672100010141000009780033
:1021f0002432ec00efff390080012000209188009c
:102200002191800030022000808f50000e003e009f
:10221000800120002412b500000678000c0646005c
:102220004067210060007e004200de0022918000b5
:102230004111dd00416721000101410000097800e2
:102240002432ec00eeff390040022000209188008b
:1022500021918000f0022000808f50000e003e008f
:10226000400220002412b500000678000c0646004b
:102270004067210060007e004300de002291800064
:102280004111dd0041672100010141000009780092
:102290002432ec00eeff390000032000209188007a
:1022a00021918000b0032000808f50000e003e007e
:1022b000000320002412b500000678000c0646003a
:1022c0004067210060007e004400de002291800013
:1022d0004111dd0041672100010141000009780042
:1022e0002432ec00eeff3900c0032000209188006a
:1022f0002191800070042000808f50000e003e006d
:10230000c00320002412b500000678000c06460029
:102310004067210060007e004500de0022918000c1
:102320004111dd00416721000101410000097800f1
:102330002432ec00eeff3900800420002091880058
:102340002191800030052000808f50000e003e005b
:10235000800420002412b500000678000c06460018
:102360004067210060007e004600de002291800070
:102370004111dd00416721000101410000097800a1
:102380002432ec00eeff3900007a2100e0b888002a
:10239000f0732100f0b88800f06d210000b98800ca
:1023a0000068210010b988004062210020b988002f
:1023b000805c210030b98800e056210040b98800d7
:1023c0006051210050b98800f04b210060b98800ad
:1023d0009046210070b988005041210080b98800e2
:1023e000203c210090b9880010372100a0b9880056
:1023f00010322100b0b98800202d2100c0b988001a
:1024000040282100d0b9880080232100e0b988004d
:10241000d01e2100f0b98800301a210000ba8800cf
:10242000a015210010ba88002011210020ba8800d0
:10243000c00c210030ba88007008210040ba880022
:102440002004210050ba8800f0ff200060ba880004
:10245000d0fb200070ba8800c0f7200080ba880046
:10246000d0f3200090ba8800e0ef2000a0ba8800e6
:1024700000ec2000b0ba880030e82000c0ba880024
:1024800070e42000d0ba8800c0e02000e0ba8800e4
:1024900020dd2000f0ba880090d9200000bb880021
:1024a00010d6200010bb8800a0d2200020bb8800de
:1024b00040cf200030bb8800e0cb200040bb88002c
:1024c000a0c8200050bb880060c5200060bb880009
:1024d00030c2200070bb880010bf200080bb880085
:1024e00000bc200090bb88000000060074b5ef001f
:1024f000a0c72500b0ab880050982500c0ab88006d
:1025000040812500d0ab8800906a2500e0ab8800b0
:1025100030542500f0ab8800303e250000ac880028
:102520009028250010ac88005013250020ac8800ae
:1025300060fe240030ac8800c0e9240040ac880074
:1025400080d5240050ac880090c1240060ac880085
:10255000f0ad240070ac8800a09a240080ac880004
:10256000a087240090ac8800f0742400a0ac880000
:1025700090622400b0ac880080502400c0ac880079
:10258000b03e2400d0ac8800302d2400e0ac8800a0
:10259000f01b2400f0ac8800000b240000ad880084
:1025a00050fa230010ad8800e0e9230020ad880038
:1025b000c0d9230030ad8800e0c9230040ad8800b9
:1025c00040ba230050ad8800e0aa230060ad880027
:1025d000c09b230070ad8800e08c230080ad880094
:1025e000307e230090ad8800d06f2300a0ad88001e
:1025f000a0612300b0ad8800b0532300c0ad8800b7
:10260000f0452300d0ad880070382300e0ad88008d
:10261000202b2300f0ad8800101e230000ae8800a0
:102620004011230010ae88009004230020ae8800e3
:1026300020f8220030ae8800e0eb220040ae880097
:10264000d0df220050ae8800f0d3220060ae8800b8
:1026500050c8220070ae8800d0bc220080ae880036
:1026600080b1220090ae880070a62200a0ae880043
:10267000809b2200b0ae8800c0902200c0ae8800cf
:1026800020862200d0ae8800c07b2200e0ae880009
:1026900080712200f0ae88006067220000af8800e1
:1026a000805d220010af8800c053220020af880058
:1026b000204a220030af8800b040220040af88009e
:1026c0006037220050af8800402e220060af8800a3
:1026d0004025220070af8800601c220080af880077
:1026e000b013220090af8800200b2200a0af88001a
:1026f000b0022200b0af880060fa2100c0af8800ad
:1027000040f22100d0af880030ea2100e0af88001d
:1027100050e22100f0af880090da210000b088007c
:10272000e0d2210010b0880060cb210020b08800ea
:10273000f0c3210030b08800b0bc210040b0880058
:1027400080b5210050b0880080ae210060b08800c4
:1027500090a7210070b08800b0a0210080b0880050
:10276000009a210090b0880060932100a0b08800fa
:10277000e08c2100b0b0880080862100c0b08800c5
:1027800030802100d0b08800007a2100e0b08800bd
:10279000f0732100f0b08800f06d210000b18800d6
:1027a0000068210010b188004062210020b188003b
:1027b000805c210030b18800e056210040b18800e3
:1027c0006051210050b18800f04b210060b18800b9
:1027d0009046210070b188005041210080b18800ee
:1027e000203c210090b1880010372100a0b1880062
:1027f00010322100b0b18800202d2100c0b1880026
:1028000040282100d0b1880080232100e0b1880059
:10281000d01e2100f0b18800301a210000b28800db
:10282000a015210010b288002011210020b28800dc
:10283000c00c210030b288007008210040b288002e
:102840002004210050b28800f0ff200060b2880010
:10285000d0fb200070b28800c0f7200080b2880052
:10286000d0f3200090b28800e0ef2000a0b28800f2
:1028700000ec2000b0b2880030e82000c0b2880030
:1028800070e42000d0b28800c0e02000e0b28800f0
:1028900020dd2000f0b2880090d9200000b388002d
:1028a00010d6200010b38800a0d2200020b38800ea
:1028b00040cf200030b38800e0cb200040b3880038
:1028c000a0c8200050b3880060c5200060b3880015
:1028d00030c2200070b3880010bf200080b3880091
:1028e00000bc200090b388000000060090dc2300ac
:1028f000a0928800b0fd2000909288002432ef0062
:1029000025f2bf0015003a0092928000a392800049
:102910002091800085f807000bf80700d1f607002a
:10292000b0928800c1928800b2928000c392800069
:1029300000002000f137240003f807005cf80700ce
:10294000229180004111dd00413721000101410049
:10295000000978002432ec00e9ff3900000006008d
:1029600090e42300a0928800b0fd2000909288009f
:102970002432ef0025f2bf0015003a009292800049
:10298000a39280002091800068f80700eef707000e
:10299000b4f60700b0928800c1928800b29280001d
:1029a000c392800010d72f00f1372400e6f707000c
:1029b0003ff80700229180004111dd0041372100de
:1029c00001014100000978002432ec00e9ff3900e0
:1029d00000000600c0122000909b88001013200009
:1029e000809b880060132000709b8800b01320003b
:1029f000609b880000142000509b88005014200029
:102a0000409b8800b0142000309b880000152000f7
:102a1000209b880060152000109b8800b0152000c6
:102a2000009b880010162000f09a88007016200085
:102a3000e09a8800d0162000d09a88003017200035
:102a4000c09a880090172000b09a8800f0172000e4
:102a5000a09a880050182000909a8800b018200092
:102a6000809a880020192000709a88008019200020
:102a7000609a8800f0192000509a8800601a20009f
:102a8000409a8800d01a2000309a8800401b20000d
:102a9000209a8800b01b2000109a8800201c20007b
:102aa000009a8800a01c2000f0998800101d2000ca
:102ab000e0998800901d2000d0998800101e200009
:102ac000c0998800801e2000b0998800001f200057
:102ad000a0998800901f2000909988001020200065
:102ae0008099880090202000709988002021200083
:102af00060998800a0212000509988003022200091
:102b000040998800c022200030998800502320007e
:102b100020998800f023200010998800802420004c
:102b20000099880020252000f0988800b02520001a
:102b3000e098880050262000d0988800f0262000d9
:102b4000c098880090272000b09888004028200076
:102b5000a0988800e0282000909888009029200004
:102b600080988800402a200070988800f02a200071
:102b700060988800a02b200050988800602c2000ce
:102b800040988800102d200030988800d02d20001b
:102b900020988800902e200010988800502f200048
:102ba0000098880020302000f0978800e030200056
:102bb000e0978800b0312000d09788008032200054
:102bc000c097880050332000b09788003034200030
:102bd000a09788001035200090978800e0352000ed
:102be00080978800d036200070978800b03720008a
:102bf0006097880090382000509788008039200026
:102c000040978800703a200030978800703b200081
:102c100020978800603c200010978800603d2000cd
:102c200000978800603e2000f0968800703f2000ea
:102c3000e096880070402000d096880080412000f7
:102c4000c096880090422000b0968800b0432000d3
:102c5000a0968800c044200090968800e04520009f
:102c60008096880010472000709688003048200029
:102c7000609688006049200050968800a04a200095
:102c800040968800d04b200030968800104d2000e0
:102c900020968800504e200010968800a04f2000fb
:102ca00000968800f0502000f095880040522000e7
:102cb000e095880090532000d0958800f0542000c3
:102cc000c095880050562000b0958800c05720005d
:102cd000a09588003059200090958800a05a2000c7
:102ce00080958800205c200070958800a05d200001
:102cf00060958800305f200050958800c0602000fb
:102d0000409588005062200030958800f0632000d4
:102d1000209588009065200010958800406720006d
:102d200000958800f0682000f0948800a06a2000d8
:102d3000e0948800606c2000d0948800306e200001
:102d4000c0948800f06f2000b0948800d0712000fb
:102d5000a0948800b07320009094880090752000a3
:102d6000809488008077200070948800707920001b
:102d700060948800707b200050948800707d200053
:102d800040948800807f200030948800a08120003b
:102d900020948800c083200010948800e0852000e3
:102da0000094880010882000f0938800508a20004a
:102db000e0938800908c2000d0938800e08e200063
:102dc000c093880030912000b09388009093200039
:102dd000a09388002432ef0021918000f0072000aa
:102de000808f500011003e002291800002014100be
:102df0004027210060007900d09088002291800057
:102e00000201410040272100600079001a12b4003d
:102e1000229180004111dd00412721000101410084
:102e2000000978002432ec00ebff390000c1b30048
:102e300078f8b70000c1b30079f8b70010c1b3004b
:102e40007af8b70010c1b3007bf8b70010c1b30027
:102e50007cf8b70010c1b3007df8b70020c1b30003
:102e60007ef8b70020c1b3007ff8b70020c1b300df
:102e700080f8b70030c1b30081f8b70030c1b300ab
:102e800082f8b70030c1b30083f8b70040c1b30087
:102e900084f8b70040c1b30085f8b70040c1b30063
:102ea00086f8b70040c1b30087f8b70050c1b3003f
:102eb00088f8b70050c1b30089f8b70050c1b3001b
:102ec0008af8b70060c1b3008bf8b70060c1b300e7
:102ed0008cf8b70060c1b3008df8b70070c1b300c3
:102ee0008ef8b70070c1b3008ff8b70080c1b3008f
:102ef00090f8b70080c1b30091f8b70080c1b3006b
:102f000092f8b70090c1b30093f8b70090c1b30036
:102f100094f8b700a0c1b30095f8b700a0c1b30002
:102f200096f8b700b0c1b30097f8b700b0c1b300ce
:102f300098f8b700b0c1b30099f8b700c0c1b300aa
:102f40009af8b700c0c1b3009bf8b700d0c1b30076
:102f50009cf8b700d0c1b3009df8b700e0c1b30042
:102f60009ef8b700e0c1b3009ff8b700f0c1b3000e
:102f7000a0f8b700f0c1b300a1f8b70000c2b300d9
:102f8000a2f8b70000c2b300a3f8b70010c2b300a4
:102f9000a4f8b70010c2b300a5f8b70020c2b30070
:102fa000a6f8b70020c2b300a7f8b70030c2b3003c
:102fb000a8f8b70040c2b300a9f8b70040c2b300f8
:102fc000aaf8b70040c2b300abf8b70050c2b300d4
:102fd000acf8b70060c2b300adf8b70060c2b30090
:102fe000aef8b70070c2b300aff8b70080c2b3004c
:102ff000b0f8b70080c2b300b1f8b70090c2b30018
:10300000b2f8b700a0c2b300b3f8b700b0c2b300c3
:10301000b4f8b700b0c2b300b5f8b700c0c2b3008f
:10302000b6f8b700c0c2b300b7f8b700d0c2b3005b
:10303000b8f8b700e0c2b300b9f8b700f0c2b30007
:10304000baf8b700f0c2b300bbf8b70000c3b300d2
:10305000bcf8b70010c3b300bdf8b70020c3b3007d
:10306000bef8b70030c3b300bff8b70040c3b30029
:10307000c0f8b70040c3b300c1f8b70050c3b300f5
:10308000c2f8b70060c3b300c3f8b70070c3b300a1
:10309000c4f8b70080c3b300c5f8b70090c3b3004d
:1030a000c6f8b700a0c3b300c7f8b700b0c3b300f9
:1030b000c8f8b700c0c3b300c9f8b700c0c3b300b5
:1030c000caf8b700e0c3b300cbf8b700f0c3b30051
:1030d000ccf8b70000c4b300cdf8b70010c4b300fb
:1030e000cef8b70020c4b300cff8b70030c4b300a7
:1030f000d0f8b70040c4b300d1f8b70050c4b30053
:10310000d2f8b70060c4b300d3f8b70070c4b300fe
:10311000d4f8b70090c4b300d5f8b700a0c4b3008a
:10312000d6f8b700b0c4b300d7f8b700c0c4b30036
:10313000d8f8b700d0c4b300d9f8b700f0c4b300d2
:10314000daf8b70000c5b300dbf8b70010c5b3006c
:10315000dcf8b70030c5b300ddf8b70040c5b300f8
:10316000def8b70050c5b300dff8b70070c5b30094
:10317000e0f8b70080c5b300e1f8b700a0c5b30020
:10318000e2f8b700b0c5b300e3f8b700c0c5b300bc
:10319000e4f8b700e0c5b300e5f8b70000c6b30037
:1031a000e6f8b70010c6b300e7f8b70030c6b300c2
:1031b000e8f8b70040c6b300e9f8b70060c6b3004e
:1031c000eaf8b70080c6b300ebf8b70090c6b300ca
:1031d000ecf8b700b0c6b300edf8b700d0c6b30046
:1031e000eef8b700f0c6b300eff8b70000c7b300c1
:1031f000f0f8b70020c7b300f1f8b70040c7b3003c
:10320000f2f8b70060c7b300f3f8b70080c7b300a7
:10321000f4f8b700a0c7b300f5f8b700c0c7b30013
:10322000f6f8b700e0c7b300f7f8b70000000600f3
:04323000ffff370065
:020000040000fa
:103234001a1200000a00000080000000241200009e
:1032440016000000800000003a1200002000000078
:10325400800000005a1200001a00000080000000e4
:1032640074120000000500008000000074170000c4
:1032740004000000800000007817000080010000b6
:083284008000000000000000c2
:00000001FF
